:10000000020CCAE4FFFE12014C600C0FEF70010EEF
:0A00100009E970F20A80EF222222B3
:06001B0080090100000055
:06002300022838C2A832D9
:10002B000237A5EFC394094005EF940E4003BF20A0
:06003B0003D38001C32283
:0E0043000216FB74FFF0A37400F0A3741D22DC
:100053000237BFE709F608DFFA8046E709F208DF4F
:10006300FA803E88828C83E709F0A3DFFA8032E3CB
:1000730009F608DFFA8078E309F208DFFA8070886E
:10008300828C83E309F0A3DFFA806489828A83E0A8
:10009300A3F608DFFA805889828A83E0A3F208DF97
:1000A300FA804C80D280FA80C680D4806980F28046
:1000B30033801080A680EA809A80A880DA80E2806C
:1000C300CA803389828A83ECFAE493A3C8C582C8C1
:1000D300CCC583CCF0A3C8C582C8CCC583CCDFE92B
:1000E300DEE7800D89828A83E493A3F608DFF9ECC7
:1000F300FAA9F0EDFB2289828A83ECFAE0A3C8C552
:1001030082C8CCC583CCF0A3C8C582C8CCC583CC78
:10011300DFEADEE880DB89828A83E493A3F208DFE7
:10012300F980CC88F0EF60010E4E60C388F0ED24B7
:1001330002B4040050B9F582EB2402B4040050AFBA
:1001430023234582239000A673BB010689828A83F9
:10015300E0225002E722BBFE02E32289828A83E483
:100163009322BB010CE58229F582E5833AF583E00E
:10017300225006E92582F8E622BBFE06E92582F82D
:10018300E222E58229F582E5833AF583E49322BBF3
:10019300010689828A83F0225002F722BBFE01F313
:1001A30022F8BB010DE58229F582E5833AF583E860
:1001B300F0225006E92582C8F622BBFE05E9258216
:1001C300C8F222EF8DF0A4A8F0CF8CF0A428CE8D36
:1001D300F0A42EFE22BC000BBE0029EF8DF084FF9D
:1001E300ADF022E4CCF875F008EF2FFFEE33FEEC10
:1001F30033FCEE9DEC984005FCEE9DFE0FD5F0E937
:10020300E4CEFD22EDF8F5F0EE8420D21CFEADF035
:1002130075F008EF2FFFED33FD4007985006D5F03A
:10022300F222C398FD0FD5F0EA22C5F0F8A3E02827
:10023300F0C5F0F8E582158270021583E038F022EC
:10024300A3F8E0C5F025F0F0E5821582700215836E
:10025300E0C838F0E822BB010A89828A83E0F5F01E
:10026300A3E022500687F009E71922BBFE07E3F556
:10027300F009E3192289828A83E493F5F0740193E8
:1002830022BB010A89828A83F0E5F0A3F02250069B
:10029300F709A7F01922BBFE06F3E5F009F31922CB
:1002A300F8BB0111E58229F582E5833AF583E8F08D
:1002B300E5F0A3F0225009E92582C8F608A6F0224A
:1002C300BBFE09E92582C8F2E5F008F222EB9FF5AF
:1002D300F0EA9E42F0E99D42F0EC6480C8648098A5
:1002E30045F022EB9FF5F0EA9E42F0E99D42F0E8EB
:1002F3009C45F022E8600FECC313FCED13FDEE13F5
:10030300FEEF13FFD8F1227401FF3395E0FEFDFCED
:10031300080808E6CF2FF618E6CE3EF618E6CD3DE0
:10032300F618E6CC3CF622ECF0A3EDF0A3EEF0A336
:10033300EFF022D083D082F8E493701274019370AB
:100343000DA3A393F8740193F5828883E473740275
:10035300936860EFA3A3A380DFD083D082F8E493F4
:100363007012740193700DA3A393F8740193F58233
:100373008883E473740293B5F0067403936860E9A9
:10038300A3A3A3A380D8E3F5F009E208B5F06BDFDC
:10039300F58067E3F5F009E608B5F05EDFF5805A0E
:1003A30087F009E608B5F052DFF6804E87F009E2E0
:1003B30008B5F046DFF6804288828C8387F009E037
:1003C300A3B5F036DFF6803288828C8387F009E4A8
:1003D30093A3B5F025DFF5802188828C83E3F5F0C4
:1003E30009E0A3B5F014DFF5801088828C83E3F570
:1003F300F009E493A3B5F002DFF40204B880878028
:10040300E9809080D4803E8015806E807E809D80C0
:10041300B7808D80A380518074803C0204C489829C
:100423008A83ECFAE493F5F0A3C8C582C8CCC583EC
:10043300CCE493A3C8C582C8CCC583CCB5F076DF22
:10044300E3DEE1807089828A83E493F5F0A3E20816
:10045300B5F062DFF4805E89828A83E0F5F0A3E67B
:1004630008B5F051DFF5804D89828A83E0F5F0A36A
:10047300E208B5F040DFF5803C89828A83E493F596
:10048300F0A3E608B5F02EDFF4802A8002805789B6
:10049300828A83ECFAE493F5F0A3C8C582C8CCC57D
:1004A30083CCE0A3C8C582C8CCC583CCB5F006DF36
:1004B300E4DEE280007FFFB5F0020F2240027F01FD
:1004C3002289828A83ECFAE0F5F0A3C8C582C8CCFE
:1004D300C583CCE0A3C8C582C8CCC583CCB5F0D551
:1004E300DFE5DEE380CF89828A83ECFAE0F5F0A3CF
:1004F300C8C582C8CCC583CCE493A3C8C582C8CC85
:10050300C583CCB5F0AFDFE4DEE280A988F0EF600D
:10051300010E4E60ABED2402B404005098F582EB5B
:100523002402B40400508E232345822390040073D5
:10053300EF4E6012EF60010EEDBB010B89828A83DF
:10054300F0A3DFFCDEFA2289F05007F709DFFCA9EC
:10055300F022BBFEFCF309DFFCA9F022E88FF0A434
:10056300CC8BF0A42CFCE98EF0A42CFC8AF0EDA437
:100573002CFCEA8EF0A4CDA8F08BF0A42DCC38256A
:10058300F0FDE98FF0A42CCD35F0FCEB8EF0A4FE4A
:10059300A9F0EB8FF0A4CFC5F02ECD39FEE43CFCDF
:1005A300EAA42DCE35F0FDE43CFC22C3E49FFFE436
:1005B3009EFEE49DFDE49CFC22FAE6FB0808E6F9B6
:1005C30025F0F618E6CA3AF622E5612455F8E60561
:1005D300612278523007027855E475F0011205BCA8
:1005E30002014C2000EB7F2ED2008018EF540F2421
:1005F30090D43440D4FF30040BEF24BFB41A00501E
:10060300032461FFE562600215620565E56570021A
:10061300056430070D7852E475F0011205BCEF0252
:100623000192020E367403D2078003E4C207F56118
:100633008B528A538954E4F562F564F565E562608B
:10064300077F2012060780F57563FFC201C200C24F
:1006530002C203C205C206C2081205D5FF700D30DF
:1006630007057F00120618AF65AE6422B4255FC28A
:10067300D5C2041205D5FF24D0B40A00501A75F070
:100683000A786230D50508B6FF0106C6A426F6200F
:10069300D5047002D20380D924CFB41A00EF5004DA
:1006A300C2E5D204020818D20180C6D20080C0D2AB
:1006B3000280BCD2D580BAD20580B47F201206074F
:1006C3002002077401B5620040F11205CCFF120647
:1006D30007020640D208D20680951205CCFB12050C
:1006E300CCFA1205CCF94A4B700679E97A087BFFFC
:1006F30020022EE562602A7E008E8275830012013D
:100703006560060EEE656370F0C2D5EBC0E0EAC02B
:10071300E0E9C0E0EE12085FD0E0F9D0E0FAD0E003
:10072300FB12014CFF60AAEBC0E0EAC0E0E9C0E0C5
:10073300120607D0E02401F9D0E03400FAD0E0FB40
:10074300E5630460DCD563D980877BFF7A08795B36
:10075300D202809C791080027908C206C208800800
:10076300D2D5790A8004790AC2D5E563047002F50B
:1007730063E4FAFDFEFF1205CCFC7B082001131293
:1007830005CCFD7B1030000A1205CCFE1205CCFF10
:100793007B20EC3382D592D55013C3E43000069FFF
:1007A300FFE49EFEE42001039DFDE49CFCE4CBF802
:1007B300C201EC700CCFCECDCCE824F8F870F380F6
:1007C30017C3EF33FFEE33FEED33FDEC33FCEB33B6
:1007D300FB994002FB0FD8E9EB300105F8D0E0C4E8
:1007E30048B201C0E00AEC4D4E4F78207B0070C246
:1007F300EAB5630040BCC0E0120861D0F0D0E0204D
:100803000104C4C0E0C4B201C0F01205F0D0F0D5B9
:10081300F0EB02064012033606DD5307575806AEC7
:100823004C06AA42075B4F07634407634906C34369
:10083300076955074D46074D45074D4709095006BA
:10084300B22D06B62E06D92B06BA2306D72008F2F8
:100853002A067248000006D13F3F3F00790AA2D51D
:10086300200314300509B910020404B9080104A2D5
:10087300D52006025001042002689202B56200509E
:1008830034C0E07F203003197F30A2027206720564
:10089300500F1208B8C202C206C205C2087F3080D8
:1008A3000F300503E9C0E0120607300503D0E0F975
:1008B300D0E0B562CC3005177F30B9100C120607B3
:1008C3007F583004077F788003B908031206073086
:1008D30002057F2D0206077F202008F87F2B2006C4
:1008E300F322920280CF286E756C6C2900D201121C
:1008F30005CC3001F8C201786230D50108F6020652
:10090300722D504349581205CC2403B4050040010D
:10091300E4900904931205F8743A1205F8D20375AA
:10092300620402075730312F30332F3038203135EE
:100933003A31303A3433000D0A000D0A496E6974B6
:100943002E2E2E000D0A253035754B20464C415373
:10095300480D0A253035754B204652414D0D0A008E
:100963002A2A4572726F72212043616E6E6F742062
:10097300636F6E6E65637420746F20434F4D004345
:100983006F6E6E656374656420746F20434F4D0012
:1009930054696D6577617665204453502D44333037
:1009A300300D0A4669726D776172653A20002052F4
:1009B300657620322E320D0A53657269616C204EC2
:1009C300756D6265723A200020204D697373696EFC
:1009D300672045746865726E657420554152542EC4
:1009E3000D0A0020204D697373696E67205361748B
:1009F300656C6C69746520554152542E0D0A0020B4
:100A030053746172742E2E2E0074656D7000766FB0
:100A13006C747300757074696D6500636F6D316F0D
:100A2300757400636F6D326F7574007374617475E0
:100A330073006C6576656C006761696E00766F6C38
:100A43003100766F6C32006672657100445350203A
:100A53004F66666C696E652E2E2E0D0A00726573E5
:100A6300657400445350204F6E6C696E652E2E2EB4
:100A73000025642064422056657220256420256386
:100A83000020256420487A00466163746F72792ED2
:100A930000476F6F64203A2047756167653A2025E8
:100AA300753A2575202D3E200046696C7465726584
:100AB30064202D3E2000426164203A20005061638F
:100AC3006B65743A20253032582025303258202562
:100AD30030325820253032580D0A000D0A466F7205
:100AE3006D617474696E672E2E2E00436F6D706C8A
:100AF3006574650D0A005772697465204661696CF7
:100B03007572650D0A0044697361626C6564204403
:100B130053502E2E2E0D0A002E0069666C6F7773CC
:100B23002575003D256C750D00FF0928FF093AFF67
:100B33000A60FF0ADEFF0AEEFF0AF98B478A48893B
:100B430049AB47AA48A94912014CFF12002E500D88
:100B530074012549F549E43548F54880E4D200ABF2
:100B630047AA48A94912014CFF642B6004EFB42D36
:100B73001BAB470549E549AA487002054814F91219
:100B8300014C642D6003D38001C39200E4F54DF55D
:100B93004CF54BF54AAB47AA48A94912014CFF1241
:100BA3000E5D505CE47F0AFEFDFCAB4DAA4CA94BE5
:100BB300A84A12055FC8ECC8EDC0E0EEC0E0EFC084
:100BC300E0AB47AA48A94912014CFF3395E0FEEF79
:100BD30024D0FFEE34FFFEE4FCFDD0E0FBD0E0FACE
:100BE300D0E0F9EB2FF54DEA3EF54CED39F54BEC42
:100BF30038F54A74012549F549E43548F5488095A7
:100C030030000AAF4DAE4CAD4BAC4A800BAF4DAE8E
:100C13004CAD4BAC4A1205AE228B478A488949AB8F
:100C230047AA48A94912014CFF12002E500D740126
:100C33002549F549E43548F54880E4D200AB47AA95
:100C430048A94912014CFF642B6004EFB42D1BAB80
:100C5300470549E549AA487002054814F912014CB1
:100C6300642D6003D38001C39200E4F54AF54BABD6
:100C730047AA48A94912014CFF120E5D5036AB47F3
:100C8300AA48A94912014CFF3395E0FEEF24D0FB9B
:100C9300EE34FFFAAE4AAF4B7C007D0A1201C6EF79
:100CA3002BF54BEE3AF54A74012549F549E43548ED
:100CB300F54880BB300006AE4AAF4B8009C3E495CC
:100CC3004BFFE4954AFE22787FE4F6D8FD75817FD9
:100CD300020D110230B2E493A3F8E493A34003F6A8
:100CE3008001F208DFF48029E493A3F85407240C6D
:100CF300C8C333C4540F4420C8834004F45680014E
:100D030046F6DFE4800B0102040810204080900DBA
:100D1300F2E47E019360BCA3FF543F30E509541F06
:100D2300FEE493A360010ECF54C025E060A840B851
:100D3300E493A3FAE493A3F8E493A3C8C582C8CACF
:100D4300C583CAF0A3C8C582C8CAC583CADFE9DEA2
:100D5300E780BE8B358A368937E4F53DF53EE53CC1
:100D6300153CAE3B7002153B4E6033AB38AA39A934
:100D73003A12014CFFAB35AA36A937053EE53EAC26
:100D83003D7002053D14F5828C83EF1201A4EF60E0
:100D9300CD7401253AF53AE43539F53980C0AB35E0
:100DA300AA36A93722434F4D003A20426175642089
:100DB30000333030003630300031323030003234DE
:100DC3003030003438303000393630300031393289
:100DD300303000333834303000353736303000258A
:100DE3003032582064656661756C74000D0A00C169
:100DF3008FC190041B00000000026800000266001F
:100E03000002730001016F00017100026C000041D8
:100E1300016B0041029B00C10E41016C00011000F7
:100E2300420000000042018B00000219000002177B
:100E3300000000EFB40A07740D120E41740A3098D3
:100E430011A899B8130CC2983098FDA899C298B804
:100E530011F63099FDC299F59922EFC394304007FA
:100E6300EF943A50028001C32212011001000000E6
:100E730040C41004800000020301010902200001A4
:100E83000100800F09040000020000000007058133
:100E930003400005070502034000050705840340DE
:100EA30000051C0309040908090C09100914091891
:100EB300091C090C09240928092C093009341203D7
:100EC300540049004D0045005700410056004500BD
:100ED30000000A0344003300300030000000900398
:100EE300D3E07010A3E0700C9003D7E07006A3E08A
:100EF3006402600312105B9003D1E0247F6013143B
:100F030060272402707D9003D5E07077A3E060151D
:100F130080719003E0E0B4040A9003D5E07004A369
:100F2300E06002805EF19880509003E0E0B4040634
:100F33009003D5E06002804B9003D6E0FFB48111AB
:100F4300E51C9003DDB403051200468002F19B808B
:100F530028EFB40211E51D9003DDB403051200462A
:100F63008002F19B8013EFB48417E51E9003DDB478
:100F730003051200468002F19B1214337402F080C1
:100F830005800012105BE51B64046008E59620E70A
:100F9300FB12147C229003DD74FFF0A37400F0A312
:100FA300741F2212167F60030210409003D1E0FFEA
:100FB3007003021040640170030210409003D3E0F9
:100FC300707B9003D5E070759003D7E0706FA3E05A
:100FD300600280699003D1E0640270619003D4E001
:100FE300705B12178E600AEF64026005EF64847011
:100FF3004CEFB48113E59620E7FB121686E59620A5
:10100300E7FB1153F51C8037EFB4021BE59620E78D
:10101300FB75960E759702E59620E7FB759614759A
:101023009780E4F51D8018E59620E7FB75960E750D
:101033009704E59620E7FB1153F51E8002115BE54B
:101043009620E7FBD18D6007E59620E7FBB14722A9
:10105300759611759740E422E59620E7FB75960E89
:10106300E4F597E59620E7FB759611759720751BB8
:1010730004229003D3E024FE602114603E14700226
:10108300215214700221632404600221BC510B74A9
:101093000EF0A3746CF0900E6C215E510B740EF085
:1010A300A3747EF0900E81E493FE900E80E4937C13
:1010B300002400FFEC3E9003DB21B69003D4E01440
:1010C300600A14605614605E2403806575280274F8
:1010D300ED2528F582E43403F583E0FFE52825E0D8
:1010E300245BF582E43403F583EFF0E52825E0245F
:1010F3005CF582E43403F583E4F00528E528B408BD
:10110300CE90035D740CF0A37403F09003DD7401BF
:10111300F0A37403F0A3745DF0801F510B740EF001
:10112300A374C1F08014510B740EF0A374D5F08036
:1011330009510B740EF0A374A5F09003DDE0FBA33B
:10114300E0FAA3E0F912014CFF9003DBE480645161
:101153000B740EF0A37487F0900E875113E4805341
:101163009003D4E0FF6481600AEF64026005EF64DA
:10117300847046EFB48111510B740EF0A37490F098
:10118300900E905113E4802B9003D4E09003DDB4D0
:10119300021074FFF0A3740EF0A37497F0900E97EF
:1011A300800E74FFF0A3740EF0A3749EF0900E9E55
:1011B3005113E4F0A3EFF08002115B9003D3E0FF3F
:1011C30064016013EF6402600EEF64036009EF646F
:1011D300046004EFB405239003D8E0FFD39003DC4D
:1011E300E09F9003DBE0940040109003D7E0700A87
:1011F300E0FE9003DBEEF0A3EFF0E51B6404600771
:10120300E59620E7FB917C229003DD74FFF0A32297
:10121300E493FF9003DB229003D1E06480701C9081
:1012230003D3E07016A3E07012A3E0700EA3E07086
:101233000AA3E07006A3E064016004115B801C90C4
:1012430003E0E0FFB40409510B12004A913304F0A8
:10125300EFB40307120F98913304F0E51B640460A5
:1012630007E59620E7FB917C22E59620E7FB759640
:101273000EE4F597E59620E7FB759691E59620E752
:10128300FB859726E51BB40511E59620E7FBE4F5FE
:10129300969003D4E0F597E4F51BE52630E20EE5DE
:1012A3009620E7FB759611E4F597F51B22E52630AA
:1012B300E419E59620E7FB759611759708E59620E6
:1012C300E7FB759611759780E4F51BE51B600261DA
:1012D3007EE52620E002617E7B017A0379D17D08D9
:1012E3007C007F201237499003D4E0FE9003D3E0C3
:1012F3007C002400FFEC3EF0A3EFF09003D6E0FE69
:101303009003D5E02400FFEC3EF0A3EFF09003D868
:10131300E0FE9003D7E02400FFEC3EF0A3EFF09053
:1013230003D2E0B40C005051901332F82828730212
:10133300135602135B02137C02136002137C021325
:101343006402136802137C02136C02137002137499
:10135300021378120EE18023120FA6801EB1CC80F7
:101363001AB100801611758012511A800EB14E8089
:101373000A913B8006918D8002115BE51B6401603D
:10138300028132E52630E1028132E59620E7FB75E2
:101393009691E59620E7FB859726E52630E4053010
:1013A300E0028132752702C39003DCE0944090038E
:1013B300DBE09400403B9003DDE0FBA3E0FAA3E015
:1013C300F97D407C007F2091C19003DEE475F040FD
:1013D30012022D9003DCE024C0F09003DBE034FF25
:1013E300F09003DAE02440F09003D9E03400F08079
:1013F3001B9003DBE0FCA3E0FDA3E0FBA3E0FAA367
:10140300E0F97F2091C1432708E4F51B9003D7E05F
:10141300FEA3E0FFA3E0B5060BA3E0B50706432751
:1014230008E4F51BE59620E7FB75961185279722BF
:10143300F09003DBE4F0A322D17F70249003D1E08A
:101443006481701C9003D3E07016A3E07012A3E0D4
:10145300700EA3E0700AA3E07006A3E064016004C9
:10146300115B8007120F98913304F0E51B6404604D
:1014730007E59620E7FB917C2275961175974075D9
:101483001B01E49003D9F0A3F0229003D1E064019F
:10149300701C9003D7E07016A3E070129003D3E0A2
:1014A300700CA3E07008A3E07004A3E06002115B7A
:1014B300E51B64046007E59620E7FBB147228C280F
:1014C3008D298B2A8A2B892CE5294528602EE596C0
:1014D30020E7FB8F96E4FFFEC3EF9529EE95285096
:1014E3001BAB2AAA2BA92C8F828E83120165F59739
:1014F300E59620E7FB0FBF00010E80DC229003D1AD
:10150300E0701D9003D5E07017A3E07013A3E070A3
:101513000FA3E0700B9003D3E07005A3E030E70264
:10152300115B751B059003D4E09003E06005740321
:10153300F080037402F0E51B64046007E59620E77E
:10154300FBB14722759611759748229003E0E0643A
:101553000260259003D1E0701F9003D5E07019A3BA
:10156300E07015A3E07011A3E0700D9003D3E07059
:1015730007A3E0D394014004115B803F9003D4E0C0
:10158300D39400402C9003E07404F0E4F51CF51DA3
:10159300E59620E7FBD186E59620E7FB7596127565
:1015A3009720D198E59620E7FB75960EE4F5978092
:1015B3000A9003E07403F0F51CF51DE51B64046059
:1015C30007E59620E7FBB14722D17F6002C16C900B
:1015D30003D1E0FF7002C16C64017002C16C90031F
:1015E300D3E06002C16C9003D5E0707D9003D7E037
:1015F3007077A3E0600280719003D1E064027069A8
:101603009003D4E07063F18E600AEF64026005EF2B
:1016130064847055EFB48117E59620E7FBD186E526
:101623009620E7FB759611759710751C03803CEFA8
:10163300B4021BE59620E7FB75960E759702E596B7
:1016430020E7FB759614759720751D03801DE5969D
:1016530020E7FB75960E759704E59620E7FB7596D4
:1016630011759710751E038002115BE59620E7FB49
:10167300D18D6007E59620E7FBB147229003E0E0B8
:1016830064042275960E7597012275960EE4F597FC
:10169300E51B640422E59620E7FB75960E7597011A
:1016A300E59620E7FB759691E59620E7FBAF97E576
:1016B3001CB4030CE59620E7FB7596117597102271
:1016C300EF30E50BE59620E7FB759611759740EF34
:1016D30030E20BE59620E7FB759611E4F5977B0165
:1016E3007A0079EB7D407C007F2191C1E59620E76C
:1016F300FB75961175970122C0E0C0F0C083C082CC
:10170300C0D075D000C000C001C002C003C004C077
:1017130005C006C007E59620E7FB759686E596208B
:10172300E7FB859723E59620E7FB759682E59620F0
:10173300E7FB859724E59620E7FB759684E59620DD
:10174300E7FB859725E52330E102F196E52330E2B7
:1017530002F1A8E52430E002516CE52430E102D126
:1017630098E52530E2031236D2E52330E002F19FFB
:10177300D007D006D005D004D003D002D001D000CA
:10178300D0D0D082D083D0F0D0E0329003D6E0FF27
:101793006481220527E52770020526220527E52710
:1017A30070020526229003E07402F0E59620E7FB21
:1017B300759601759701E4F51B751C03751D0322CE
:1017C3001219D5E4F531E4F530AF301231F91231A5
:1017D30051E4755801F557F556F5557F90123226A9
:1017E3001219708F2E1219708F2FE52E12033618CF
:1017F3002841181943181E44181E48181149182364
:1018030080181E8D18238E1830FF00001830753293
:1018130000753380801C753201800D75320280089B
:1018230075320480037532087533008005E4F532A0
:10183300F533D3E5339400E53294004012AF301210
:1018430031F97F5011C3AF301231F97F0111BFE578
:101853003025E024E1F582E43403F583E532F0A397
:10186300E533F0123D00E4F0A3F0AF30EFD3940082
:10187300401DEF25E024DFF582E43403F583E0FC2B
:10188300A3E0FD123D00EC8DF012022D1F80DD055B
:1018930030E530C3940350030217CC31D50531E54D
:1018A30031C39402500D9003E9E07002A3E070038A
:1018B3000217C922F148E4FF11C3E4FF11C3E4FF97
:1018C30030F9FDC2FF8FA330FFFD228B378A3889A1
:1018D30039746A2FF8E67003FEFF2231D5F1487F91
:1018E3005511C37F02316E8F3B31708F3CE53CF461
:1018F300B53B07E53BD3953A40087F1831D3E4FE67
:10190300FF22E4F53EE4F53FF540F53CE53CC395A5
:101913003B502431708F3D7E00E5402FFF753F0023
:101923008F40AB37AA38A939853C82758300E53DE2
:101933001201A4053C80D531708F3CE540F4B53CE1
:10194300067F0611C3800D7F1511C3053EE53EC317
:10195300940540B1E53EB4050B7F1811C37F181100
:10196300C3E4F53B31D5AF3B7E002211C3E4FF1145
:10197300C3AFA3228F3C8D3D746A2FF8E67002FF3C
:101983002231D5AF3C11B7AF3CF1487FA311C3AFB0
:101993003D316E8F3D31D5E53D7002F1EBE53D7094
:1019A30002F1EBAF3D228F3E746A2FF8E67002FF1F
:1019B3002231D5AF3E11B7AF3EF1487FA411C331F9
:1019C30070800F53903B43A03DD2954390447F06D4
:1019D30011C353903B43A03DD295227E007A0179F7
:1019E3002B123CA77A0079EB123CA77F0E7D007B7C
:1019F300017A01796D1205337E007F107D007B0132
:101A03007A01797B120533E4786EF69000E9F0A34E
:101A1300F07A09793DD1A57FFF7870EFF6F1D6789A
:101A230072760212282FC007C006123681755A003B
:101A33008F5BD058D0597555FF755609755747F1C7
:101A430041120628F141D1B7F141122898E4F51269
:101A5300E4F511AF12F18ABFFF0AAF12F18AEFF476
:101A630060058000751101E5117BFF70067A097925
:101A73006380047A097982D1B7E5122432FF1239DF
:101A83009C7BFF7A09793AD1B70512E512D3940109
:101A930040BE1233039000F1E0FF123057AD077FD1
:101AA300011239AA123B973177AD077F021239AA87
:101AB300C2901232C8C20DC20CD28290010674FFCA
:101AC300F0123CF77BFF7A097993D1B7900B2CD1B5
:101AD300AC7BFF7A0979B1D1B77B017A0379EFD176
:101AE300A7E56B70087BFF7A0979CBD1B7E56A70FC
:101AF300087BFF7A0979E6D1B77A0A7902D1A5780A
:101B030079E6FE08E6FF7874667003EE18666029CE
:101B13007873A60608A607787BE6FE08E6FF7C0036
:101B23007D0B1201C6900177EEF0A3EFF07877E614
:101B3300FF08E6A3CFF0A3EFF0C3787AE694141876
:101B4300E69400500281F1E4F608F6787106E69413
:101B530002405DE4F6786F06900187123D0E240182
:101B6300123B84900187123B8F30E408786D06E6C0
:101B730018700106123D694003E004F090029BE0F7
:101B8300D394004010E004F0D3940A40087872E63E
:101B930054FEF6E4F0300E1290016CE0D394004052
:101BA30005E014F0800AC20E800690016C740AF0FE
:101BB300309104C2918002D2919000F3E020E402BC
:101BC30081D390012BE030E10281D3AF100510EFF8
:101BD3001203361C13011C1E021C29031C34041C93
:101BE30060051C3F061C60081C550A1C600B1C6E1C
:101BF3000C1C600E1C60101C60121C55141C60151C
:101C03001C6E161C7B171C88181C931B00001CA63B
:101C13007BFF7A0A790C900179807E7BFF7A0A79BF
:101C23001190017780737BFF7A0A7917900187807F
:101C3300147BFF7A0A791E90017B80097BFF7A0A65
:101C4300792690017F123D0EF5518E508D4F8C4EAB
:101C5300804A7A0A792E9000F3F1C8803F7BFF7A9D
:101C63000A79359000EF123CE880317BFF7A0A79DC
:101C73003B90016DF1CA80247BFF7A0A7940900181
:101C83006FF1CA80177A0A7945900170F1C8800C08
:101C93007BFF7A0A794A9000E9123CE87F0112340B
:101CA30045802DE510C3941C4003E4F5109000001B
:101CB300E0FEA3E0FF123406900001E02408F09058
:101CC3000000E03400F0C3E094204004E4F0A3F00B
:101CD300D3786DE694B418E69400401EE4F608F653
:101CE300123D39F07B107D107F01F19F800CF14193
:101CF3007DB01228F9F1411228EC7970E778726609
:101D03007005123D69403890016BE0FFD3940040A9
:101D130025EF75F00684AFF07401A807088002C3AD
:101D230033D8FCFFF1D690016BE0C3943C4010E440
:101D3300F07870F680097872E67870F6FFF1D620B5
:101D4300820F9000EDE04404F1407DB012246780DF
:101D5300189000EDE054FBF0123D24F0300D0A7BA7
:101D6300FF7A0A794FD1B7C20DF1417DB012203904
:101D7300F1411228EC120018122FEE4002610212F8
:101D83002FF68F11E511C394005002C13390000A5E
:101D9300E511F0E4A3F078027C007D017B017A0079
:101DA3007903FE7F07120126900008E511F0E4A3F2
:101DB300F140D1B778047C007D01900B32E4123CF2
:101DC300D4F97E007F0512050FEF60026102900BCC
:101DD30032123CD4F9E4755101F1CF7F011234453D
:101DE3007E00123D401220061232A090028BE4F0D6
:101DF300A3740CF0900289E4F0A3740CF090028DAC
:101E0300E4F0A3740EF0900293E4F0A37480F090D6
:101E13000291E4F0A37480F0E4A3F0A3F0A3F0A391
:101E23007483F0A37401F0A3742CF012276261028F
:101E3300E4FF8F33787FE6D39400403CD20A787F67
:101E4300E6FF18E6FED39F5007E408F618F680264F
:101E5300C3EE9F787EF6F58275830074DD2FF9E477
:101E63003402FA7B0178DD7C027D017E00AF8212B1
:101E73000126E4787FF6C20A787EE6C3947E400E9C
:101E8300787FE670B7300BF8C20BD29980F2787E78
:101E930012288EF583E533F0300B04C20BD299AFD1
:101EA30033227BFFD1B7900B2FE493FB740193FA9A
:101EB300740293F98B4B8A4C894DEA494B6011129A
:101EC30000038E4E8F4F1234A9AD4FAC4E1238CC57
:101ED30090012FE0FF900104E06F705912381A8EC1
:101EE3004E8F4FD3E54F9409E54E94004006754E4F
:101EF30000754F09D3E54F9400E54E9400403190AF
:101F030000EDE04401F07B017A0079FAAD4F12381D
:101F130041900105E54FF090012FE0C3947E5008F6
:101F2300E004900104F0800D9001047401F0800539
:101F3300E4900105F09000EDE054FEF022F07B0107
:101F43007A00790A2231D5EF146006047005C2A421
:101F530022C2A02231D54390447F05123589EF7008
:101F630004C20F802031708F2EE52EB4FF04C20F00
:101F7300801331C6439044532EF9532E7F7F0111B2
:101F8300C3AF2E11C321D5746A2FF8E67002FF2266
:101F930031D5F1487FA511C3317021D58F358D36E9
:101FA3008B37746A2FF8E6601BAF35F18A8F38AF31
:101FB30035F148E536F45238E53742387FAA11C384
:101FC300AF3831D3227BFFE0FFE48F51F550F54F5B
:101FD300F54E2253903B43A03DD29553A1CF75A21A
:101FE3007FC2A511C3D2A522AF3C31A98F3D227F69
:101FF300031231F97F501231F47F011218C3E4FF49
:102003000218C38F4D8E4C8D4B8C4A7F031231F9CE
:102013007F061231F4854D58854C57854B56854ABA
:10202300557F521232261219D51231517F031232C3
:10203300AFEF20E0F7221228B2E4FD90012DE0FF7C
:102043009000F9E06F7002411890012CE014B4186D
:10205300004002411590205F123D19730220B20225
:1020630022150220CA0220D402213802213D022176
:102073007B0220DE0220F00220BE02212D02215627
:102083000221020221140222150221B30220A70217
:1020930020C402214702219B02220F02216B02214D
:1020A300EE0221FCE4900108F0900106F04115F1E5
:1020B3001E7F01F145F11E7F028073F11E7F0780B1
:1020C3006DF11E7F09806790013DE0FD1236188097
:1020D3005F90013DE0FD1236278055F1E67F05F163
:1020E30045900173E0FCA3E0FD7F06804190017100
:1020F300E0FCA3E0FD7F05F145F1E67F06802F902C
:10210300013DE0FF1230579000F1EFF0FD7F0180B9
:1021130014123D61121977123D611219779000F282
:10212300EFF0FD7F021239AA8006F1E67F08F14540
:10213300122F0D41151232C84115123D39F07B1093
:102143007D108008123D39F07B307D307F01121FF6
:102153009F411590013DE09000F36006E04480F05C
:102163004115E0547FF041159003CDE0900109F053
:102173009001077401F04115123CF790012C741182
:10218300F0122F0DE4F5311231510531E531C394CD
:102193006440F443EF90807A90013DE06009D20CF3
:1021A30043A404C282806BC20CD28253A4FB80621C
:1021B3007B017A01793D900136E0F5567F01D1DE4E
:1021C300900183E0F8A3E0F9A3E0FAA3E0FB900118
:1021D30036E0FFE4FCFDFEEB2FFFEE3AFEED39FDAA
:1021E300EC38FC90018312032A80277A01796D7FF2
:1021F3000E123CB3122FE580197A01797B7F1012FE
:102203003CB3E054EFF0E04420F0800690016BE033
:1022130004F0123CF790013BE0FF900108E06F707F
:102223000241B7E4FFFE7D109001379131402B301E
:10223300820241D1900137123C56123D2FF53112E3
:102243003CDE85314B7A017909754F017550017573
:10225300510990013C12325680527FFF7EFF7D0F61
:102263007C0090013791327020900B2C123CD48B60
:10227300388A39F53A90013CE0753B00F53C7B0127
:102283007A017909120D568023E4FFFE7D0FFC903D
:10229300013791324016900137123C86123C771277
:1022A3003CC47A01790990013C1233FE90013BE072
:1022B300900108F090012EE0FF900106E06F70029C
:1022C300812BE47D10912C500261CD308216900158
:1022D30006E064FE7002812B74FEF07BFF7A0B79BB
:1022E30009021EB7900131123C56123D2FF531FF02
:1022F300FEFD91467013900B35121EADE4F515F1FA
:10230300EF900B38121EAC8066E47D059144700F8C
:10231300900B35121EADE4F515FFFE7D05804D9142
:1023230041700B900B35121EAD123D59803E914109
:10233300700B900B35121EAD123D59802F7E80120B
:102343003D4091477010900B35121EADE4F515FF1B
:102353007E807D048016E4FFFE7D0691467010901A
:102363000B35121EADE4F515FFFE7D06FC11067B51
:10237300FF7A0B791B121EB70515E515D39446405A
:1023830006121EA9E4F515123CDE85314B7A01795C
:102393003D754F0175500175513D900135E0F55282
:1023A3007F03122F2F123CDE85314B852E4F852F55
:1023B30050853051900135123256915312050FEF6B
:1023C3006050900B3B121EAC8048E47D0F912C4073
:1023D30038900131123C86123C77123CC47A017961
:1023E3003D900135E0754C00F54D122F87AE33AFAC
:1023F3003491609001351233FE915312050FEF6053
:1024030006900B3B121EAC8009E4FFFE7D0E912E5D
:10241300400990012EE0900106F022E4FFFE7D0DBD
:10242300912E90010674FDF022FFFE900131FCE035
:10243300F8A3E0F9A3E0FAA3E0FBC30202E6E47D1C
:1024430004FFFEFCAB34AA33A932A831C30202E66F
:10245300900135E0FF7E00783D7C017D01AB2EAA23
:102463002FA930221228B2E4FD300D02A1417BFFD7
:102473007A0A7966121EB7D20D300C02A1351235D5
:10248300CB120019121FF2F1681236897555FF75C8
:10249300560A75577490016DE024E8F559E434FF4A
:1024A300F5589003CD123D477F4430E1027F508FB2
:1024B3005C91601206289160121EB77D1A7F01128B
:1024C30035EE7D1A7F0212361A12362BE4F513F518
:1024D30014F54EF54D754C04F54B7A007932F54FF2
:1024E300755000755132123299754E01754D007554
:1024F3004C04754B007A007931754F0075500075A7
:102503005131123299C3E53294A0E531940F502B27
:102513007555FF75560A755784AE31AF329000E991
:10252300EEF0A3EFF08E58F55991601206289160F2
:1025330080067BFF7A0A798B121EB7121EA9300C14
:1025430002C1DDE51475F01484E5F07026123689B6
:102553009003CEE09000ED30E006E04408F0800404
:10256300E054F7F09003CBE0FFA3E09000EFCFF04F
:10257300A3EFF00514E514D394C85002C1DDE4F5CC
:10258300149003C2E09000F4F0E07002C1DDE513A3
:1025930054F0FFE054F06F603653130FE054F042F1
:1025A30013E51354F0C4540FF5317872E654E3F68F
:1025B300E531D3940C4006E64410F68012E531D39E
:1025C30094097872E640054408F680034404F6E56E
:1025D30013540FFF9000F4E0540F6F7002C1DD53EA
:1025E30013F0E0540F42137B017A0079F51233B5EF
:1025F3009000F5E0FF121E359000F6E0FF121E3545
:102603009000F7E0FF121E359000F8E0FF121E3530
:1026130090017B123B7890017B12032A753601757A
:1026230037007538CE7B017A0079F5122DA9EF605A
:102633005A7872E64401F690029B7401F07555FFD7
:1026430075560A7557949000CEE0F558A3E0F559F6
:10265300A3E0F55AA3E0F55B91601206289160129E
:102663001EB7123D50123559EF70079000F3E0305A
:10267300E70E123D50A3E0FCA3E0FD123A5C802E6E
:102683007BFF7A0A79AC121EB78023123D24F07BBC
:10269300FF7A0A79B9121EB79000F3E030E70FF121
:1026A30037E4FFD1DE123B7590017F12032A755583
:1026B300FF75560A7557C09000F5E0755800F55937
:1026C300A3123D47755C00F55DA3E0755E00F55F01
:1026D30091601206289160121EB7228B538A548987
:1026E30055746A2FF8E660321219D5121F487F5AC3
:1026F3001218C37F011218C3AF568016AF56155672
:10270300EF6014AB530555E555AA547002055412F6
:102713002FCD1218C380E51219D52290013DE0FD9B
:102723007C00227F01D1DE7B017A0079F5755604A6
:102733007F01D1DE7B017A0079F575560422AC4323
:10274300AD448F478C488D491232A0E54725E024DC
:1027530087F582E43402F583E548F0A3E549F012F6
:1027630034FC122F2F1234FC12325B90028AE09059
:10277300016DF090028EE090016EF0900291E0FF07
:10278300A3E0900171CFF0A3EFF0900293E0FFA3D9
:10279300E0900173CFF0A3EFF0900296E09000EB8E
:1027A300F0900297E0FFA3E0900175CFF0A3EFF064
:1027B30090029AE09000ECF0222010037FFF221297
:1027C30019D51235E7BF01047FC080027FC21218FA
:1027D300C31235E7121970EF541FFFC3741F9FFF15
:1027E3000219D590013DE0FCA3E0FD22E4F538F5A4
:1027F30037F536F535E4FFFE7D04FCAB38AA37A97F
:1028030036A835C31202E65022AF38AE37AD36AC28
:1028130035122006E42538F538E5373480F537E4FA
:102823003536F536E43535F53580CA229003E5E0D3
:10283300FEA3E0FF22C0E0C083C082C0D075D008F1
:1028430030981DC298787DE6C3943E500DE6062469
:102853009DF582E43402F583800390029CE599F0B0
:1028630030991FC299200A18797EE7D3787F964062
:1028730009118EF583E0F5998002D20BD20980020B
:10288300D20BD0D0D082D083D0E032E60624DDF55F
:1028930082E434022211B212246012014C600F054B
:1028A30030E5307002052FF1CD121E3580E9228B01
:1028B3002E8A2F89302211B28D31E4FF121F8AEF45
:1028C300F46025EF30E321122460E53114F53AE496
:1028D300FF1218CE8F16122460D1B4E516D39400DC
:1028E3004006122460121EB7227DB011B97B007A14
:1028F300007900021EB711B28D31E4F5327F011267
:102903001F8A8F35E535F47002414EE53520E30229
:10291300414E30E402414E122460E53114F53A7F12
:10292300011218CE8F33E533D3940050024136128F
:102933002460D1B4D390018CE09400D1654005E4C8
:10294300F53421F8E4F534E534C3953340024136D8
:10295300122460853482758300120165F53554F0C5
:10296300FFBFF01685334BAD34D16E8F33E535643D
:10297300F660079000F3E04410F0E535240CB40B47
:10298300004002413290298F123D1973022A270217
:102993002A1F0229B70229F80229EF0229E6022990
:1029A300DC0229D20229C90229C00229B09000F30E
:1029B300F1E580939000F3E054EFF0808A9000F308
:1029C300E04401F080819000F3E054FEF0214AE4FA
:1029D300786CF608F6D290214AE4786CF608F6C2D1
:1029E30090214A9000F3E04420F0214A9000F3E064
:1029F30054DFF0214AC3E5339534F533AB2E7E0023
:102A0300E5302534F9EE352FFA753900753A00753E
:102A13003B33514FE5342533F533214A9000F3E03E
:102A2300440280069000F3E054FDF0F10D214A05C5
:102A330034214AE533D394004006122460121EB7B2
:102A43000532E532C3940A50022100228B368A37BD
:102A53008938D1416046640D6042916D12014CD3B7
:102A630094004038D15F5034D141FF90018BE4751D
:102A7300F001120243FCD1BD3CF583EFF0C003C06B
:102A830002C001916D12014CF54BD001D002D0036D
:102A9300E4FDD16E916DEF12019280B690018BE04F
:102AA3007002A3E0701290018B75F001120243FED5
:102AB300D1BD3EF5837420F0D3D15F4006E4F0A38B
:102AC3007413F090018CE024BAF582E43400F583AA
:102AD300E4F0D141FF640D6007EF640A60028152A4
:102AE300E490018BF0A3F0C003C002C001916D120A
:102AF300014CF54BD001D002D003E4FDD16E916DB2
:102B0300EF120192D1C6B10C12014CFF6008643D73
:102B13006004D15380F0EF643D60028152AB3C0509
:102B23003EE53EAA3D7002053D14F9E4120192B15F
:102B33000C12014CB42004D15380F4120B3E8F4489
:102B43008E438D428C41D1C6B10C12014CB420048A
:102B5300D15380F4120C1C8E3F8F40C3E53F942069
:102B6300505AE5407803CEC313CE13D8F97A0079CF
:102B73004512334AE540F1DC8002C333D8FCF54605
:102B8300AF44AE43AD42AC41EC4D4E4F7007E5460A
:102B9300F452458004E5464245E540AE3F7803CE16
:102BA300C313CE13D8F9F1D47B007A007945754C61
:102BB30000754D01F187AF40AE3F8047E540853F4B
:102BC300F012035C2C0B20002C1320012BE360017B
:102BD3002BEA60022BF160032C02600400002C52EC
:102BE300AD441236188068AD4412362780617F01E8
:102BF3001227417F02122741F10D1232C88050AED5
:102C030043AF4412340680477E007F147DFF800665
:102C13007E007F147D007B017A0079BA120533E4CC
:102C2300F53FF540C3E53F94045024E42540FFE518
:102C33003F3402FE7B017A0079BA754C00754D145E
:102C4300F18774142540F540E4353FF53F80D59175
:102C53006D12014CAB36AA37A938F582758300E4AF
:102C63000201A4E5F08FF0120284AB39AA3AA93B22
:102C730022D1A59000021201655401C454F0B10C95
:102C830075F000B109C003C002C001120259FDACC6
:102C9300F0916DD14A543F7806C333CE33CED8F981
:102CA300D1ACD001D002D003B106C003C002C00131
:102CB300120259FF916DD1DBD001D002D00391668E
:102CC300900002120165543EFFE4C313FEEF13FFAD
:102CD300B10CD1E5C003C002C001120259FDACF032
:102CE300916D9000031201657E00543F7805C33354
:102CF300CE33CED8F9D1ACD001D002D003EE8FF0D1
:102D0300020284EE8FF0120284AB3CAA3DA93E225C
:102D1300D1A5D14A547F7806C333CE33CED8F9FF39
:102D2300B10CB106C003C002C001120259FF916D7C
:102D3300D1DBD001D002D0039166D14A5480780709
:102D4300CEC313CE13D8F9FFB10CD1E5C003C00233
:102D5300C001120259FD916D90000212016525E038
:102D6300FFE43345F0FEED4FFFD001D002D003EE78
:102D73008FF0120284AB3CE53E2402F9E4353DFAC0
:102D8300C003C002C001120259FD916D90000312ED
:102D93000165540325E045F0FFEDD001D002D003D7
:102DA300CF8FF00202848B338A348935AB36AA374E
:102DB300A93874FFF5F0120284AB36AA37A938900C
:102DC300000274FFF5F01202A3D107D1F6EF4E60B3
:102DD30007B1FEB1137F0122D107123BEAEF4E6028
:102DE30007B1FE91747F0122D107123C20EF4E60A0
:102DF30007B1FED10E7F01227F002285363C853745
:102E03003D85383EAB33AA34A93522D1A5900001C4
:102E1300D1D012014C540F7C002FFFEC35F0B10CD4
:102E23009168900003D1D0900002120165540F2FD6
:102E3300FFEC35F0B10C9000028FF00202A3AB3629
:102E4300AA37A93802014C9000011201657E0022C5
:102E53007401253EF53EE4353DF53D2290018CE0BD
:102E6300941390018BE064809480228B478A488975
:102E730049154BEDC3954B501BEDF582758300A3AC
:102E8300AB47AA48A9491201658D827583001201D7
:102E9300A40D80DFAB47AA48A949854B82D1B6AFC1
:102EA3004B228B398A3A893B22FFEC4EFEED4FFFD2
:102EB300228F82758300E40201A474BA25F0F5829F
:102EC300740022753C01753D00753EBA22120165FE
:102ED300540F75F00AA4FF2212014C543FFDEF4D2D
:102EE300FF22900002EE8FF01202A3E92402F9E41C
:102EF3003AFA2212014C54C0FFBFC00A123B9FEFA3
:102F03007004FE7F0122E4FEFF227B017A0079EB4D
:102F1300754C00754D40E4FFFEF187E4F54BF54A2F
:102F2300F549F5487F021231C41235158F4A85528F
:102F330053AF521552EF6041AF4A1231F97F061277
:102F430018C3AF4A1231F9784B12030A8F588E57C0
:102F53008D568C557F02123226AB4F0551E551AA8F
:102F6300507002055014F912014CFF1218C3AF4AF6
:102F73001232AFEF20E0F780B853903B43A03DD22D
:102F830095AF53228E478F488B498A4A894B300F1E
:102F930038E54D454C60321219C6439044AD48ACF8
:102FA300477F021234C0E54D154DAE4C7002154CEF
:102FB3004E6013AB49054BE54BAA4A7002054AF133
:102FC300CD1218C380E01219D52214F912014CFF57
:102FD300222400FFEE3402FE225407FF7401A807E7
:102FE3000822E054DFF0E04410F022787DE6D3704D
:102FF30001C322787DE670037FFF2290029DE0F5F6
:103003002E787D16E66013E6FF7E00789D7C027DB8
:10301300017B017A02799E120126AF2E22C28EC253
:10302300AB759810D29C758D30538EF07F25115758
:10303300758BFF53890F438920D209D20BC20AE44F
:10304300787DF608F608F6C299C298D2ACD2BCD203
:1030530099D28E228F35538EF4E53524FC602124DA
:10306300FB602224F7602324ED602724DA60252403
:10307300B5602624B5602724DF7028758D30800D58
:10308300758D988008758DCC8003758DE6438E020F
:10309300801A8012758DB28010758DD9800B758D55
:1030A300E68006753525758D64438E01AF35225351
:1030B300D9BF759003B13153903B43A03DD29531B5
:1030C3003191B0438004E4787BF608F67879F6080A
:1030D300F691E591D211201217C3121F5731607B6D
:1030E300017A0379EF754F007550057F007E0171FA
:1030F30059752D0274ED252DF582E43403F583E033
:10310300FFD3947F5006EFC3942050117E007F05B8
:103113007D307B017A0379EF1205338007052DE5B6
:103123002DB407D0E49003F4F0D1360219DE43B294
:1031330083E4F5B943B98043B9C03151E5B97004AB
:103143007F0180027F00EF20E5F2E4F5A922E4FF8E
:10315300FE0FBF00010EBE01F8BFF4F5221219D510
:10316300E4F52FE4F52E3151AF2E121F487FA5B1A0
:1031730089EF7009746A252EF8E4F6800C12197031
:103183008F30746A252EF87601746A252EF8E6606E
:1031930012AF2E121F484330017FAA1218C3AF305B
:1031A3001218C3052EE52EC3940240BA1219D50591
:1031B3002FE52FC394025008E56A7004E56B60A302
:1031C300228F4731F97F061218C3AF4731F9854B78
:1031D30058854A578549568548557F20512653902F
:1031E3003B43A03DD2953151AF4751AFEF20E0F8BB
:1031F300221218C37F0353903B43A03DD295EF1493
:1032030060111460121460131460142404701343C7
:10321300908422439080224390C0224390402243D3
:103223009044221218C3AF58AE57AD56AC558F5CBD
:103233008E5B8D5A8C5978101202F71218C3AF5C4B
:10324300AE5BAD5AAC5978081202F71218C3AF5CE3
:103253000218C3E0F5527F0331F9854E58854D5767
:10326300854C56854B557F035126855253AF5215D6
:1032730052EF6017121970AB4F0551E551AA507008
:1032830002055014F9EF12019280E253903B43A0E0
:103293003DD295AF53227552017F0380BB91FC5100
:1032A3005B7F007E007D057C000220068F5431F990
:1032B3007F051218C31219708F5453903B43A03DDE
:1032C300D295AF5422D2A7E4F547F54831510548CA
:1032D300E54870020547C39458E5476480948240EB
:1032E300EBC2A7E4F547F54831510548E5487002BC
:1032F3000547C394B0E5476480948440EBD2A7228A
:10330300B115515B9000F3E0B4FF117B017A0079B2
:10331300EB754F00755040E4FFFE71599000F3E0E8
:10332300B4FF02E4F09000F3E05402F0E04440F014
:10333300121F38E49000F9F0900105F0A3F090011A
:1033430008F09000F4F0222400FFEE3402FE7B002C
:10335300754F007550018B4C8A4D894EAD07AC06F5
:10336300E4F551F552300F06E550454F7004E4FE85
:10337300FF221219D54390447F0391C0E5501550A5
:10338300AE4F7002154F4E601B121970AB4C054EB9
:10339300E54EAA4D7002054D71AF0552E55270021C
:1033A300055180D81219D5AE51AF522214F9EF024C
:1033B30001928B338A3489359003C4E0FF0535E5E8
:1033C300357002053471AF9003C671F5AA347002EB
:1033D300053471AF9003C871F5AA347002053471D6
:1033E300AF9003CA71F5AA347002053414F9EF02E1
:1033F3000192E0FFAB330535E53522E0754F00F56B
:103403005061598E478F48E5487803CEC313CE13D6
:10341300D8F9122FD47B007A00794971537555FF7F
:1034230075560B75571D8547588548597B017A009A
:1034330079D21206287B017A0079D2E549121FCB93
:103443007F018F4A8B4B8A4C894DE54AB401079023
:10345300012BE020E0489000DD74AAF0A3F091A2D4
:10346300755602AF4A1226DE91A91200038F5691B8
:10347300A9AF4A1226DE7555FF75560B755726857B
:10348300515B85505A854F59854E5891A212062893
:1034930091A21200038F5691A2AF4A1226DE227B1D
:1034A300017A0079DD22AB4BAA4CA94D2275A2F01B
:1034B30075A140E4F5F8D2F9D2F8C2FF228C538DFE
:1034C300541218C3E553FF1218C3AF540218C3753F
:1034D300D10775BB1E75BA1F75BCFC75E8C243E600
:1034E3000822E4F5C8538ECF75CB9D75CAF474FFDB
:1034F300F5CDF5CCD2ADD2CA22E4F54EF54D754CDF
:1035030005F54B754F017550027551877552147F40
:103513000322E4F54EF54DF54CF54B7A0079EB7546
:103523004F017550007551EB7552407F022275D6DD
:10353300FF75D5FF75D48C75F3FD75F2FF43F18CE0
:1035430043A4C153A4F375A5C775A6FD75E103E4B0
:10355300F5E243E240228E338F3453331FE534AE1A
:10356300337803CEC313CE13D8F97A007935714A71
:10357300E534122FDC8002C333D8FCFF55356F7F4F
:103583000160027F0022E4F533F53430F9FDC2FF18
:103593008FA320FF1A0534E53470020533FFAE33E1
:1035A300E4FCFD7B507AC3F9F8D31202D050E3AEAA
:1035B30033AF34E4FCFD7B507AC3F9F8D31202D065
:1035C30050037F00227F0122D2101219D5B1E77F69
:1035D30080B189EF7004C2108007B1E77FA0121891
:1035E300C30219D55390FB439004228D4730102416
:1035F3001219D5E547541FFEC3741F9E541FF54788
:10360300B1E7BF0104AF478005E5474440FF121807
:10361300C31219D5227F01B1EE7F011227BC90019D
:103623006FEFF0227F02B1EE7F021227BC90017090
:10363300EFF022E59620E7FB759601759708E5966E
:1036430020E7FB759607759707E59620E7FB7596C8
:1036530009759707E59620E7FB75960B7597077530
:10366300D7E0E59620E7FB75960F75978043E60252
:10367300D2AFE59620E7FB759601759701227F0887
:10368300200F027F002220822B1219D5C295E4F568
:1036930033AF337E00D1B8E53325E024C1F582E4AE
:1036A3003403F583EEF0A3EFF00533E533C3940859
:1036B30040DFD29522AD07AC06AF04EC121972AE0F
:1036C30007AF05121972AD07AF06EFFEEDFF22E457
:1036D300FFE59620E7FB75960E759702E59620E7C2
:1036E300FB759694E59620E7FBAE97E51DB4030CB6
:1036F300E59620E7FB75961475972022EE30E60BCE
:10370300E59620E7FB759614759780E59620E7FB11
:10371300759696E59620E7FBAF97EF6440600DE55D
:103723009620E7FB759616759710800E7B017A013C
:10373300792B7D407C007F22F149E59620E7FB75DC
:103743009614E4F597228C288D298B2A8A2B892CB1
:10375300E5294528604B8F964396C0E4FFFEE52993
:1037630024FFFDE52834FFFCC3EF9DEE9C501BE5D1
:103773009620E7FBAB2AAA2BA92C8F828E83E59791
:103783001201A40FBF00010E80D4E4F596E5962044
:10379300E7FBAB2AAA2BA92C8F828E83E597120114
:1037A300A422C0E0C0D075D000C000787A06E61825
:1037B300700106C2CFD000D0D0D0E032C0E0C0D07C
:1037C30075D000C000C001C005C006C007E5BBB48A
:1037D3001E1BAFBEEFFEADBDED7806CEC313CE13F9
:1037E300D8F97978F7EE19F775BB098019AFBEEFF1
:1037F300FEADBDED7806CEC313CE13D8F9797CF7B1
:10380300EE19F775BB1EC2EDD007D006D005D00167
:10381300D000D0D0D0E032C3E518951AE51795193A
:10382300400BE518951AFFE5179519FE22C374FAA4
:10383300951ACFE49519CF2518CF3517FE228B5053
:103843008A5189528D53C374FA951AF555E4951923
:10385300F554C3E5559553E5549400400AAF537EA0
:103863000011B4AD508029AE54AF5511B4AD501210
:103873000126C3E5539555FFE49554FEE5522555BE
:10388300F9E5513554A801FCAD507B017A01798DDE
:103893001201267E00E51A2553FFEE351911C48C5B
:1038A300198D1A111AC3EF944AEE94005002C20EF6
:1038B30022748D251AF9E43401FA7B01A852AC5124
:1038C30022FE7C007DFA0201D88B508A5189528CEA
:1038D300538D543173501E3191C3EF9554EE95536C
:1038E3005013051AE51A70020519FFAE1911C58C9C
:1038F300198D1A80E23173400675530F7554FFC357
:1039030074FA9518F556E49517F555C3E55695548D
:10391300E55595534008AE53AF54317D8026AE55DF
:10392300AF56317D120126C3E5549556FFE55395F5
:1039330055FEAB50E5522556F9E5513555FA788DCC
:103943007C017D01120126E5182554FFE517355347
:1039530011C48C178D18111A8E538F54D3E55494B8
:103963004AE55394004008D20E90016C740AF02289
:10397300C3E55494FAE553940022748D2518F9E4B1
:103983003401A801FC7D01AB50AA51A95222111A9E
:10399300C374F99FFFE49EFE228F4B7B007A00796C
:1039A3004B7D017C0001CC8F358D367BFF7A0D7901
:1039B300A8121EB7E5352430FF319C7BFF7A0D79C1
:1039C300AC121EB7E53612033639EB0139F302396F
:1039D300FB043A03093A0B123A13253A1B4B3A23D9
:1039E300963A2BE100003A337BFF7A0D79B4805687
:1039F3007BFF7A0D79B8804E7BFF7A0D79BC8046C8
:103A03007BFF7A0D79C1803E7BFF7A0D79C68036C4
:103A13007BFF7A0D79CB802E7BFF7A0D79D08026C0
:103A23007BFF7A0D79D6801E7BFF7A0D79DC8016B9
:103A33007555FF75560D7557E27558008536595102
:103A4300551206285155121EB77BFF7A0D79EF02E6
:103A53001EB77B007A007937228E338F348C358DF5
:103A63003653331F5335079000F3E030E142EF54F0
:103A73003F44C0F537E534AE337806CEC313CE13D7
:103A8300D8F9547FFFAE36EEC433333354804FF549
:103A930038E535C313E53613F539E535C313540358
:103AA300F53A5155719F8F3BE53B54FC423A80797F
:103AB300D3E5349463E53394004042E534543F4402
:103AC30040F537E534AE337806CEC313CE13D8F9B9
:103AD300543F4440F538E533C45401FFAE36EE2578
:103AE300E0543E4F44C0F539E536AE357805CEC3D4
:103AF30013CE13D8F9543F44C0F53A802CAE33AFFC
:103B030034716EEF540F4403F537AE33AF34716E37
:103B1300ED540F4403F538716AEF540F4403F5393C
:103B2300716AED540F4403F53A71971219775155A1
:103B3300755604E4FF1226DE717590017F718F3094
:103B4300E422753BAB7B007A00793B755601122763
:103B5300261227267F011226DE90018371789001B9
:103B63008312032A7F0122AE35AF367C007D0A0221
:103B730001D890017FE0FCA3E0FDA3E0FEA3E024D5
:103B830004FFE43EFEE43DFDE43CFC2212032A90E4
:103B930000F3E0229000F2E0FDE4FF228B3C8A3D3B
:103BA300893EE4F53FFFFE122D0C8F828E831201B6
:103BB30065FDE4FBFAE53FC313F53FED30E0034356
:103BC3003F80EDC313FDE53F30E103633F9A0BBB39
:103BD30000010AEB64084A70DC0FBF00010EEF64BA
:103BE300044E70C3AF3F2212014C54C0644070298D
:103BF30090000112016554C06440701D90000212D0
:103C0300016554C0FFBFC01190000312016554C089
:103C1300FFBFC0057E007F0122E4FEFF2212014C9C
:103C2300547064307029900001120165547064303F
:103C3300701D9000021201655470FFBF3011900097
:103C4300031201655470FFBF30057E007F0122E43B
:103C5300FEFF22E0FCA3E0FDA3E0FEA3E0F5348E2B
:103C6300338D328C31C39400F534E5339400F5334E
:103C7300E5329410F532E5319400F531E534F5344D
:103C8300E53322E0FCA3E0FDA3E0FEA3E0F5348EE0
:103C9300338D328C319400F534E5339400F533E5FC
:103CA30032940F227F407D007B011205337E002278
:103CB300781B7C017D017B017E001201269000EDC3
:103CC30022541FF533E4F532F531AE33AF347B01C3
:103CD3002293FB740193FA7402932285344E853345
:103CE3004D85324C22E0FEA3E0FFE48F518E50F568
:103CF3004FF54E2290012DE09000F9F022E530259A
:103D0300E024E7F582E43403F58322E0FCA3E0FD3D
:103D1300A3E0FEA3E02275F003A4C58325F0C583C9
:103D2300227872E654FEF6E490029B22F533E532E4
:103D33005407F532E4229000F3E054CF227F007D54
:103D4300047C0022E0755A00F55BA3E0229000CECC
:103D5300E0FEA3E0FF22E4F515FFFE7D04229001BF
:0E3D63003DE0FDE4FF2290016BE0D3940022CE
:00000001FF
